:020000040000FA
:020000000528D1
:080008000900831681018C013F
:100010008E018E15FF30850086009F0183128B01B3
:100020008501860190019201970198019F01831635
:100030008601831223203C2056206D208620A32099
:10004000B620D0201A2886010614E2208614061055
:10005000E22006158610E22086150611E22006161B
:100060008611E22086160612E22006178612E2208A
:1000700086170613E22008008601E2208617E22098
:1000800006178613E22086160613E220061686124D
:10009000E22086150612E22006158611E22086145B
:1000A0000611E22006148610E22008008601E220F4
:1000B0000614E22006150610E22006160611E220BC
:1000C00006170612E22006160613E220061506128F
:1000D000E22006140611E220080086010614E22040
:1000E0008614E2200615E22086150610E220061688
:1000F0008610E22086160611E22006178611E220FD
:100100008617061286120613E2200800860186175B
:10011000E2200617E2208616E22006168613E22069
:1001200086150613E22006158612E22086140612B2
:10013000E22006148611E2200611E2208610E22059
:100140000610E22008008601E2200614E220861450
:10015000E2200615E2208615E2200616E220861629
:10016000E2200617E2208617E2200800E220FF3096
:100170008600E2208601E220FF308600E220860130
:10018000E220FF308600E2208601E220FF30860078
:10019000E2208601E220FF308600E220860108008E
:1001A000E2200610E2208610E2200611E2208611ED
:1001B000E2200612E2208612E2200613E2208613D5
:1001C000E22008000F30C000C00BE72808003230E2
:1001D000C200C20BEC28E428C10BEC28E9288614E5
:1001E0000610E22086158610E22086168611E2208F
:1001F00086178612E22086168613E220861586125E
:0A020000E22086148611E2200800B7
:02400E00103E62
:00000001FF
